:020000040000FA
:02000000702866
:08000800D400030E8301D500B2
:1000100086308100D603031D5C280830D600DA083C
:10002000031DDA03DB08031DDB03DC08031DDC030F
:100030005D085E0403192028DE035E090319DD0351
:100040005F086004031930285F08633C031D2C28F7
:1000500060089C3C03193028E00360090319DF03A2
:10006000E108031DE103E208031DE203E308031DA9
:10007000E3036408650403194128E50365090319CE
:10008000E40366086704031951286608633C031DEE
:100090004D2867089C3C03195128E7036709031999
:1000A000E603D708031DD7035808590403195C2831
:1000B000D90359090319D8030B11550E8300D40E27
:1000C000540E09006C0872233108E0003208DF008A
:1000D0000800710872233108E7003208E6000800C2
:1000E000AF013A270830D600A001A101DA01DB01F7
:1000F000DC01DD01DE01E101E201E301E401E501F2
:10010000D701D201D801D9017224E001DF01E70152
:10011000E601221C6220221C69202A278511042264
:100120000B22A501061A9F280C30AF003A27A50321
:10013000031D9228182737242723342570281827D1
:10014000372404220B222C23AF013A273A273A27DF
:100150003A273A273A2737248316C730810083127B
:1001600086308100A0308B00CD20D420E1201421E6
:10017000082122212921221C322156215F216621BA
:100180007321A6219A21B421BB21221CC421E8217C
:10019000B8220D222A22AB22B428F121031D080027
:1001A0002019080020150800F12103190800201D5E
:1001B0000800201CDF286808DA006908DB0020112D
:1001C0000800201D0800201A080020180800201B25
:1001D0000800FF212014A016DB08031DF7286B0878
:1001E00072238B133108DE003208DD008B174808BC
:1001F000C2005C27031908008B13221C62208B1796
:10020000221C922B5F086004031D080092236220C9
:10021000201B0800201C080020190800DA08031D14
:100220000800042220100800201B0800201C0800E1
:100230005D085E04031D0800042220172010A01290
:10024000DA010800201F0800201D08006A08DC00F1
:100250000800201F080020190800DC08031D080002
:10026000201308005F086004031D0800201B08001D
:10027000201A08004708C2005C27031908008B13E6
:1002800062208B1720188D2BFF212014A0168D23A0
:10029000DB08031D53296B0872238B133108DE0022
:1002A0003208DD008B176808DA0008002018080003
:1002B000DB08031D0800DE01DD01A0120800F721A4
:1002C000031D0800A0190800A0150800F721031954
:1002D0000800A01D0800A01C71296D08E1006E082F
:1002E000E200A0110800A01D0800A01A0800A01834
:1002F0000800A01B08000622A0142016E208031D17
:100300008929700872238B133108E5003208E40054
:100310008B174A08C2005C27031908008B13221CA4
:1003200069208B17221C922B66086704031D0800A6
:1003300092236920A01B0800A01C0800A019080037
:10034000E108031D08000B22A0100800A01B0800F4
:10035000A01C080064086504031D08000B22A017F8
:10036000A0102012E1010800A01F0800A01D080035
:100370006F08E3000800A01F0800A0190800E308A8
:10038000031D0800A013080066086704031D080089
:10039000A01A0800A01B08004908C2005C27031926
:1003A00008008B1369208B17A0188D2B0622A01430
:1003B00020168D23E208031DE529700872238B1394
:1003C0003108E5003208E4008B176D08E1000800F1
:1003D000A0180800E208031D0800E501E40120124E
:1003E00008002119FD290508220610390800A11965
:1003F000FD290508220620390800031108002118EC
:100400000800861D0614080006100800A118080040
:10041000061C86150800861108002A271022182FAE
:10042000061D0800F321A104F921A104060E0F39CD
:10043000A9007208D700D7080319080006191B2A5B
:100440004C3052078400513C031C080029088000EE
:10045000D20A08005708031D0800A21C342A5208BB
:10046000043C0319442A8A2A5208023C0319822AAE
:100470005208063C03194E2A8A2A4C0ECD044E0E11
:10048000CF04500ED10408003D2210309F220319E2
:100490005E2A13309F220319782A8A2A3D225108A6
:1004A000D30010308E2203195E2A10309F220319C8
:1004B0005F2A13308E220319782A8A2A221373089E
:1004C00072233108D9003208D8002110A11021115F
:1004D000A1118B13211E702A221D702AE001DF0159
:1004E000A11E762AA21D762AE701E6018B178A2A29
:1004F00016305C27A20004220B222114A11421151E
:10050000A1158A2A4C0E4D045302031D8A2A221F6C
:100510008A2A782AD2012112A1120800A9005C2798
:100520004D02031D0800A90A29085C274F02031D7C
:100530000800290A5C275102031D08000800A900D1
:100540005C274D02031D0800A90A29085C274F02F9
:10055000031D08000800221F080058085904031D45
:10056000080004220B222114A1142115A115080052
:10057000003021232030A01A3E30A300682402302E
:100580002123203020195230A30068240330212376
:100590005D08B2005E08B1008223492307302123A1
:1005A0005F08B2006008B100822349230B30212389
:1005B0005B08B1003F230D30212320302018543038
:1005C000201B5330A30068240E302123B2015A08A7
:1005D000201B5C08B1003F23403021232030201A2B
:1005E0003E30A3006824423021232030A01952302D
:1005F000A3006824433021236408B2006508B100D9
:1006000082234923473021236608B2006708B100DE
:10061000822349234B3021236208B1003F234D3010
:1006200021232030A0185430A01B5330A30068248D
:100630004E302123B2016108201B6308B1003F2323
:10064000080085108038A300682485140800003055
:1006500021239430A700302B003021238330A700C2
:1006600039238A01003803190800A3006824A70A67
:10067000302B07308A0027088200003008005723FB
:100680003608303EA30068243708303EA3006824B3
:10069000080057233408303EA30068243508303E54
:1006A000A30068243608303EA300682408003830D0
:1006B00084005E235E235E235E2308001030A500C5
:1006C000B3010310B10DB20DB30DF63033070318AB
:1006D000B3000318B10AA503031D612B840333087B
:1006E00080000800B1006430A900B2010830A50004
:1006F0000310311C7D2B2908B207B20CB10CA50BDD
:10070000782B08000830AA00AB012A08B107013095
:100710000318B2072B08B20708004308C0004508B9
:10072000C100972B4408C0004608C100972BB8228F
:10073000AF013A273A27A21B572E42085C2703191C
:10074000BE2BA800203C031DAA2B16241624162419
:10075000C20A9D2B28082F3C031DBB2BE830A800A4
:10076000D223D223D223E030A800D223D2231624CE
:100770001624C20A9D2BBF23C20A9D2B08004130BC
:100780002802031CE22B193C031CD12B193CD93E37
:10079000DB23A8008A01D223D223D223D22316241A
:1007A00016240800A80DA90DA80D290D0339A900CC
:1007B000031DFC2B0800A80007308A0028088200CF
:1007C000003008003030A802031CF62B0A30280243
:1007D0000318F62B0A3EF33EDB23A8008A01F72319
:1007E000F723F723F723F723162416240800A9017B
:1007F000A80D0318A90AFC2B0330291C0130A50001
:100800004108A600CF3083169F008312400822249F
:10081000C03083169F00831240082224A603031DC4
:10082000022CA503031D002C162408004108A60075
:10083000000040082224000040082224A603031DD3
:10084000182C0800AF0000000000000000000000AD
:100850000000000000000000000000000000000098
:10086000000000000000AF03031D232C0800AF01AF
:100870003A2785103030A4005C240530AF003A27B9
:100880003030A4005C246430AF0054273030A40022
:100890005C242030A4005C242830A30068240130AC
:1008A000A30068240230AF003A270630A300682472
:1008B0000C30A3006824080006080F3924048600C1
:1008C00000000514000005102830AF005427080070
:1008D0002308F039A4005C2423080F39A400A40ED7
:1008E0005C24080005305C27EB0004305C27E8003E
:1008F00006305C27EC0007305C27E90008305C27F5
:10090000EA000A305C27F00009305C27ED000B306C
:100910005C27F1000C305C27EE000D305C27EF0007
:100920000E305C27F2000F305C27F30016305C2796
:10093000A20000305C27C30001305C27C5000230F4
:100940005C27C40003305C27C6001730C700A9002D
:10095000A903A90A29085C27031DA92C290AC80094
:10096000A90A29085C27031DB02C290AC900A90A75
:1009700029085C27031DB72C290ACA00A90A2908DF
:100980005C27031DBE2C290ACB000800A7003923D1
:100990008A010038031908001825A70AC72C5C270C
:1009A000A400240ED72418252408D724182D0F3985
:1009B000A3000A3023020318E12C3030A3072308D8
:1009C00008003730A307230808005C27B100B201F4
:1009D00057233508303E18253608303E182537088D
:1009E000303E18250D3018250A30182D3130F92CDD
:1009F000323018253A30182D20250319FC2C1825E3
:100A0000281BA81228080800840020252808A9000F
:100A1000182529080D3C0319162D291BA912290890
:100A20008000840AA703031D052D0800800108002B
:100A3000A8008316981C1A2D831228089900080014
:100A400025250319202DA8000800180806390319C8
:100A50002E2D1A08181218160315080003158C1EDF
:100A600008001A08031108009430C624F224A530A7
:100A7000C624FA241630A9000530A500A90A2908C1
:100A80005C270319452D18253E2DA50303194B2D71
:100A90002C3018253E2DF2243F3018250530A500B6
:100AA000163083169B008312FC240D3C03196C2D19
:100AB00083169B0A831228082C3C0319632D2808EF
:100AC0000D3C031D652DA801A50328086227A50874
:100AD00003196C2DFC24582DF224AA30C624F224CC
:100AE00046301825F6240030E524392653301825E1
:100AF000F6240130E524392646301825F824023042
:100B0000E524392653301825F8240330E524392606
:100B1000B330C62431301825F224C930C624F62457
:100B20000430E5243926CC30C624F6240530E524EB
:100B30003926CF30C624F6240630E5243926D230B3
:100B4000C624F6240730E5243926D630C624F624F8
:100B50000830E5243926B330C62432301825F22473
:100B6000C930C624F8240930E5243926CC30C624FF
:100B7000F8240A30E5243926CF30C624F8240B3077
:100B8000E5243926D230C624F8240C30E524392651
:100B9000D630C624F8240D30E5243926B930C624D1
:100BA000F224543018254D301825FA240E30E5244F
:100BB00039264F30182546301825FA240F30E52401
:100BC0003926C430C624F6241030CF241130CF2467
:100BD0001230CF24F22410300426F224C430C6246C
:100BE000F8241330CF241430CF241530CF24F2242E
:100BF00013300426F224BF30C624FA241630CF2442
:100C0000F2241A26F224080083169B0083123F3038
:100C100018252126031908002A08622783169B0A33
:100C2000831221262A08622783169B0A8312212613
:100C30002A08622F3F3018252126031908002A08A8
:100C4000622FFC240D3C031908002D26280EAA0053
:100C5000FC242D26AA04031108003030A8020A3013
:100C600028020318352E28080800F930A80728089C
:100C700008003F30182541260319402E2A08622714
:100C8000F22CFC240D3C0319080028080F397223AC
:100C90003108AA00FC240F39B1000A30A9007523DD
:100CA0003108AA07FC240F39AA07031108000530F0
:100CB000BC00B901BA014B30A500D726A50B5D2EAB
:100CC000FF30BD00BE00D7264B08A7000630A500A8
:100CD00084266030BF00B2260630A5008426E130AD
:100CE000BF00B2260330BF00B226F030BF00B226EC
:100CF00042085C27BF003F080319812EB226C20AB2
:100D0000782EA526D726080027085C27BF000310E9
:100D1000BF0DB226A70AA503031D842E08000130CB
:100D2000BE06BE0C031C9D2EBE0D0314BD0CBE0CD6
:100D30000830BE060430BD060800000000000000B8
:100D4000BE0D0310BD0CBE0C08003D08A5003E08FA
:100D5000BF00FF30BF06B2262508BF00FF30BF0628
:100D6000B22608000830BB00BF0C0318C22EE426D0
:100D7000912600000000000000000530BC00BB0B05
:100D8000B42E0800BC030319CA2EE4268F26BB0B21
:100D9000B42E08000314E4260530AF0054270310D6
:100DA000E4268F260530BC00BB0BB42E08007E3035
:100DB000BF000830BB00BF0CE42600000530AF00C8
:100DC0005427BB0BDB2E08000318E82E0130BA06AF
:100DD0003A18012F1C30B80039080F397227C03873
:100DE0009F000C30AF005427B90AB80BEC2E39081D
:100DF0000F397227C0389F000130AF005427B90A5D
:100E000008000F30B80039080F397227C0389F002A
:100E10001B30AF005427B90AB80B032F39080F391C
:100E20007227C0389F001030AF005427B90A08005D
:100E30008316343085000630860024309800413017
:100E40009900C0309F0083129030980007309F00B7
:100E500085110800831634308500F6308600023094
:100E60009800C0309F0083120030980007309F0028
:100E700085150800E330B00000000000000000000D
:100E80000000000000000000000000000000000062
:100E900000000000000000000000B003031D3C2F14
:100EA000AF03031D3A2F08000000000000000000FF
:100EB000AF03031D542F080083169B001C141A084F
:100EC000831208008C1383169A001C1555309D0060
:100ED000AA309D009C1483128C1F6C2F83161C1546
:100EE00083120800820708340B340D340E340F349B
:100EF0000E340D340B34083405340234013400341C
:100F000001340234053452344534503443344F34C0
:100F10004E342D343434203420344A345334313474
:100F200052345334563400345334453454345534E5
:100F3000503420344D344F3444344534203420343C
:100F400020342034203420340034433441344C34B1
:100F50004C340034203443345734203454344F3428
:100F60004E3445340034203450344F3452345434E9
:100F700000342034443454344D34463400344D3439
:100F80004F344434453400345034413453345334B2
:100F90000034483441340034543458340034493433
:100FA00044340034523445345334003453344C34D4
:100FB0000034B034EA34EE34E8348034AE34F834FB
:100FC000AA34A034BF34EC34BA34F034E034FC3406
:100FD000BE34FB34B834A834C034AC34AB34BC3485
:100FE000EB34EF34FA34F8347834383418340834C5
:0A0FF00000348034C034E034F034E3
:02400E00423F2F
:104200009C0028009C0019000A00120006001E00F5
:1042100063000A00120006001E0063000A0012007C
:1042200049008600460073008800490001004400F0
:10423000450020004A005200310057004E000000A7
:104240004A005200310057004E0000004400450073
:1042500020004A005200310057004E0000004A0082
:104260005200310057004E0000005200450050003F
:1042700043004F004E004A005200310057004E00EC
:04428000200000001A
:00000001FF
